 s3c_lcd

 Timestamp is 4be8ce34 (Tue May 11 12:25:40 2010)

 Preferred load address is 10000000

 Start         Length     Name                   Class
 0001:00000000 00000004H .CRT$XCA                CODE
 0001:00000004 00000004H .CRT$XCZ                CODE
 0001:00000008 00000004H .CRT$XIA                CODE
 0001:0000000c 00000004H .CRT$XIZ                CODE
 0001:00000010 00000004H .CRT$XPA                CODE
 0001:00000014 00000004H .CRT$XPZ                CODE
 0001:00000018 00000004H .CRT$XTA                CODE
 0001:0000001c 00000004H .CRT$XTZ                CODE
 0001:00000020 00000124H .rdata                  CODE
 0001:00000144 00000024H .rdata$debug            CODE
 0001:00000168 0000107cH .text                   CODE
 0001:000011e4 00000014H .xdata                  CODE
 0001:000011f8 00000014H .idata$2                CODE
 0001:0000120c 00000014H .idata$3                CODE
 0001:00001220 00000068H .idata$4                CODE
 0001:00001288 0000000cH .idata$6                CODE
 0001:000012a0 0000009dH .edata                  CODE
 0002:00000000 00000068H .idata$5                DATA
 0002:00000068 00000008H .data                   DATA
 0002:00000070 0000001cH .bss                    DATA
 0003:00000000 00000150H .pdata                  DATA

  Address         Publics by Value              Rva+Base       Lib:Object

 0000:00000000       ___safe_se_handler_count   00000000     <absolute>
 0000:00000000       ___safe_se_handler_table   00000000     <absolute>
 0001:00000000       __xc_a                     10001000     corelib0:crt0init.obj
 0001:00000004       __xc_z                     10001004     corelib0:crt0init.obj
 0001:00000008       __xi_a                     10001008     corelib0:crt0init.obj
 0001:0000000c       __xi_z                     1000100c     corelib0:crt0init.obj
 0001:00000010       __xp_a                     10001010     corelib0:crt0init.obj
 0001:00000014       __xp_z                     10001014     corelib0:crt0init.obj
 0001:00000018       __xt_a                     10001018     corelib0:crt0init.obj
 0001:0000001c       __xt_z                     1000101c     corelib0:crt0init.obj
 0001:0000003c       ??_C@_1M@DMCDIEDK@?$AAP?$AAK?$AAM?$AA1?$AA?3?$AA?$AA@ 1000103c     s3c_lcd_wince.obj
 0001:00000048       ??_C@_1CG@OAKGANKB@?$AA?2?$AAP?$AAo?$AAw?$AAe?$AAr?$AAV?$AAR?$AA?2?$AAP?$AAV?$AAR?$AAK?$AAe?$AAr?$AAn?$AAe?$AAl?$AA?$AA@ 10001048     s3c_lcd_wince.obj
 0001:00000070       ??_C@_0BJ@JODNLMDK@PVRGetDisplayClassJTable?$AA@ 10001070     s3c_lcd_wince.obj
 0001:0000008c       ??_C@_1DI@JINNBDNE@?$AA?$FL?$AAS?$AA3?$AAC?$AA_?$AAL?$AAC?$AAD?$AA?3?$AAE?$AAR?$AAR?$AA?$FN?$AA?5?$AAh?$AAd?$AAc?$AA?5?$AAi?$AAs?$AA?5?$AAN?$AAU?$AAL?$AAL?$AA?$AN?$AA?6?$AA?$AA@ 1000108c     s3c_lcd_displayclass.obj
 0001:000000c4       ??_C@_0CC@GJKALKLI@?$FLSGX?$FN?5FrameBuffer?5Address?5?$DN?50x?$CFx@ 100010c4     s3c_lcd_displayclass.obj
 0001:000000e8       ??_C@_0DC@DHAEFINM@?$FLS3C_LCD?$FN?5IOCTL_HAL_QUERY_DISPLA@ 100010e8     s3c_lcd_displayclass.obj
 0001:0000011c       ??_C@_0CA@MBCDNJHC@?$FLS3C_LCD?$FN?5Bit?5Per?5Pixel?5Error?$CB?6?$AA@ 1000111c     s3c_lcd_displayclass.obj
 0001:0000013c       ??_C@_07NMHLBFLJ@S3C_LCD?$AA@ 1000113c     s3c_lcd_displayclass.obj
 0001:00000168       ZwOpenFileWrap             10001168 f   s3c_lcd_wince.obj
 0001:000001b0       AllocContigMemoryMapping   100011b0 f   s3c_lcd_wince.obj
 0001:00000228       FreeContigMemory           10001228 f   s3c_lcd_wince.obj
 0001:00000230       DCH_Init                   10001230 f   s3c_lcd_wince.obj
 0001:00000248       DCH_IOControl              10001248 f   s3c_lcd_wince.obj
 0001:00000250       DCH_Deinit                 10001250 f   s3c_lcd_wince.obj
 0001:00000260       DCH_Open                   10001260 f   s3c_lcd_wince.obj
 0001:00000264       DCH_Close                  10001264 f   s3c_lcd_wince.obj
 0001:0000026c       AllocKernelMem             1000126c f   s3c_lcd_wince.obj
 0001:00000270       FreeKernelMem              10001270 f   s3c_lcd_wince.obj
 0001:00000274       OpenPVRServices            10001274 f   s3c_lcd_wince.obj
 0001:000002bc       ClosePVRServices           100012bc f   s3c_lcd_wince.obj
 0001:000002cc       GetLibFuncAddr             100012cc f   s3c_lcd_wince.obj
 0001:00000930       Deinit                     10001930 f   s3c_lcd_displayclass.obj
 0001:000009f0       GetBufferDimensions        100019f0 f   s3c_lcd_displayclass.obj
 0001:00000abc       Init                       10001abc f   s3c_lcd_displayclass.obj
 0001:00000d60       CreateFileW                10001d60 f   coredll:COREDLL.dll
 0001:00000d70       VirtualFree                10001d70 f   coredll:COREDLL.dll
 0001:00000d80       VirtualCopy                10001d80 f   coredll:COREDLL.dll
 0001:00000d90       VirtualAlloc               10001d90 f   coredll:COREDLL.dll
 0001:00000da0       FreePhysMem                10001da0 f   coredll:COREDLL.dll
 0001:00000db0       ActivateDevice             10001db0 f   coredll:COREDLL.dll
 0001:00000dc0       CloseHandle                10001dc0 f   coredll:COREDLL.dll
 0001:00000dd0       DeviceIoControl            10001dd0 f   coredll:COREDLL.dll
 0001:00000de0       NKDbgPrintfW               10001de0 f   coredll:COREDLL.dll
 0001:00000df0       ReleaseDC                  10001df0 f   coredll:COREDLL.dll
 0001:00000e00       ExtEscape                  10001e00 f   coredll:COREDLL.dll
 0001:00000e10       GetDC                      10001e10 f   coredll:COREDLL.dll
 0001:00000e20       KernelIoControl            10001e20 f   coredll:COREDLL.dll
 0001:00000e30       DllMain                    10001e30 f   corelib0:dllmain.obj
 0001:00000f4c       _DllMainCRTStartup         10001f4c f   corelib0:pegdmain.obj
 0001:00001044       _cexit                     10002044 f   corelib0:cexit.obj
 0001:00001060       _initterm                  10002060 f   corelib0:crt0dat.obj
 0001:00001094       _cinit                     10002094 f   corelib0:crt0dat.obj
 0001:000010c8       __security_init_cookie     100020c8 f   corelib0:seccinit.obj
 0001:00001124       malloc                     10002124 f   corelib1:COREDLL.dll
 0001:00001134       free                       10002134 f   corelib1:COREDLL.dll
 0001:00001144       strcmp                     10002144 f   corelib1:COREDLL.dll
 0001:00001154       printf                     10002154 f   corelib1:COREDLL.dll
 0001:00001164       memcpy                     10002164 f   corelib1:COREDLL.dll
 0001:00001174       memset                     10002174 f   corelib1:COREDLL.dll
 0001:00001184       strncpy                    10002184 f   corelib1:COREDLL.dll
 0001:00001194       _XcptFilter                10002194 f   corelib1:COREDLL.dll
 0001:000011a4       __C_specific_handler       100021a4 f   corelib1:COREDLL.dll
 0001:000011b4       __security_gen_cookie2     100021b4 f   corelib1:COREDLL.dll
 0001:000011c4       DisableThreadLibraryCalls  100021c4 f   coredll:COREDLL.dll
 0001:000011d4       TerminateProcess           100021d4 f   coredll:COREDLL.dll
 0001:000011f8       __IMPORT_DESCRIPTOR_COREDLL 100021f8     coredll:COREDLL.dll
 0001:0000120c       __NULL_IMPORT_DESCRIPTOR   1000220c     coredll:COREDLL.dll
 0002:00000000       __imp_CreateFileW          10003000     coredll:COREDLL.dll
 0002:00000004       __imp_VirtualFree          10003004     coredll:COREDLL.dll
 0002:00000008       __imp_VirtualCopy          10003008     coredll:COREDLL.dll
 0002:0000000c       __imp_VirtualAlloc         1000300c     coredll:COREDLL.dll
 0002:00000010       __imp_FreePhysMem          10003010     coredll:COREDLL.dll
 0002:00000014       __imp_ActivateDevice       10003014     coredll:COREDLL.dll
 0002:00000018       __imp_CloseHandle          10003018     coredll:COREDLL.dll
 0002:0000001c       __imp_DeviceIoControl      1000301c     coredll:COREDLL.dll
 0002:00000020       __imp_NKDbgPrintfW         10003020     coredll:COREDLL.dll
 0002:00000024       __imp_ReleaseDC            10003024     coredll:COREDLL.dll
 0002:00000028       __imp_ExtEscape            10003028     coredll:COREDLL.dll
 0002:0000002c       __imp_GetDC                1000302c     coredll:COREDLL.dll
 0002:00000030       __imp_KernelIoControl      10003030     coredll:COREDLL.dll
 0002:00000034       __imp_malloc               10003034     corelib1:COREDLL.dll
 0002:00000038       __imp_free                 10003038     corelib1:COREDLL.dll
 0002:0000003c       __imp_strcmp               1000303c     corelib1:COREDLL.dll
 0002:00000040       __imp_printf               10003040     corelib1:COREDLL.dll
 0002:00000044       __imp_memcpy               10003044     corelib1:COREDLL.dll
 0002:00000048       __imp_memset               10003048     corelib1:COREDLL.dll
 0002:0000004c       __imp_strncpy              1000304c     corelib1:COREDLL.dll
 0002:00000050       __imp__XcptFilter          10003050     corelib1:COREDLL.dll
 0002:00000054       __imp___C_specific_handler 10003054     corelib1:COREDLL.dll
 0002:00000058       __imp___security_gen_cookie2 10003058     corelib1:COREDLL.dll
 0002:0000005c       __imp_DisableThreadLibraryCalls 1000305c     coredll:COREDLL.dll
 0002:00000060       __imp_TerminateProcess     10003060     coredll:COREDLL.dll
 0002:00000064       \177COREDLL_NULL_THUNK_DATA 10003064     coredll:COREDLL.dll
 0002:00000068       __security_cookie          10003068     corelib0:seccinit.obj
 0002:0000006c       __security_cookie_complement 1000306c     corelib0:seccinit.obj
 0002:0000007c       _exitflag                  1000307c     corelib0:cexit.obj
 0002:00000080       __onexitend                10003080     <common>
 0002:00000084       __onexitbegin              10003084     <common>
 0002:00000088       _pRawDllMain               10003088     <common>

 entry point at        0001:00000f4c

 Static symbols

 0001:0000036c       OpenDCDevice               1000136c f   s3c_lcd_displayclass.obj
 0001:00000468       CloseDCDevice              10001468 f   s3c_lcd_displayclass.obj
 0001:00000470       EnumDCFormats              10001470 f   s3c_lcd_displayclass.obj
 0001:000004d4       EnumDCDims                 100014d4 f   s3c_lcd_displayclass.obj
 0001:00000558       GetDCSystemBuffer          10001558 f   s3c_lcd_displayclass.obj
 0001:00000574       GetDCInfo                  10001574 f   s3c_lcd_displayclass.obj
 0001:000005ac       GetDCBufferAddr            100015ac f   s3c_lcd_displayclass.obj
 0001:00000620       CreateDCSwapChain          10001620 f   s3c_lcd_displayclass.obj
 0001:000007cc       DestroyDCSwapChain         100017cc f   s3c_lcd_displayclass.obj
 0001:0000080c       SetDCDstRect               1000180c f   s3c_lcd_displayclass.obj
 0001:00000814       SetDCSrcRect               10001814 f   s3c_lcd_displayclass.obj
 0001:0000081c       SetDCDstColourKey          1000181c f   s3c_lcd_displayclass.obj
 0001:00000824       SetDCSrcColourKey          10001824 f   s3c_lcd_displayclass.obj
 0001:0000082c       GetDCBuffers               1000182c f   s3c_lcd_displayclass.obj
 0001:000008a0       SwapToDCBuffer             100018a0 f   s3c_lcd_displayclass.obj
 0001:000008c8       SwapToDCSystem             100018c8 f   s3c_lcd_displayclass.obj
 0001:000008dc       ProcessFlip                100018dc f   s3c_lcd_displayclass.obj
 0001:00000e50       _DllMainCRTStartupHelper   10001e50 f   corelib0:pegdmain.obj
 0001:00000f7c       doexit                     10001f7c f   corelib0:cexit.obj
